:0200000480007A
:100000006F00C004732F2034930F8000630AFF0336
:10001000930F90006306FF03930FB0006302FF038A
:10002000170F0080130F0FFE63040F0067000F000F
:10003000732F203463540F006F004000136E9E53E3
:10004000171F00002320CFFD6FF09FFF732540F1A5
:100050006310050073251030635805000F00F00F82
:10006000130E100073000000130E00009702000032
:10007000938282F973905230735020307350303035
:1000800073504030970200809382C2F7638C020065
:10009000739052109302B01A739022307323203061
:1000A000E39E62F873500030970200009382420191
:1000B00073901234732540F173002030130E20002A
:1000C000930000001301100063962000631AC02BF8
:1000D0006316C001E39E20FE6314C02B130E300094
:1000E000930010001301000063962000631AC029DA
:1000F0006316C001E39E20FE6314C029130E400066
:100100009300F0FF1301100063962000631AC027CC
:100110006316C001E39E20FE6314C027130E500037
:10012000930010001301F0FF63962000631AC025AE
:100130006316C001E39E20FE6314C025130E600009
:100140009300000013010000639420006314C001B9
:100150006318C023E39E20FE130E7000930010006E
:1001600013011000639420006314C001631AC021BE
:10017000E39E20FE130E80009300F0FF1301F0FFBA
:10018000639420006314C001631CC01FE39E20FE23
:10019000130E9000130200009300000013010000F2
:1001A0006390201E1302120093022000E31652FEF9
:1001B000130EA000130200009300000013010000C2
:1001C00013000000639E201A130212009302200005
:1001D000E31452FE130EB00013020000930000005F
:1001E000130100001300000013000000639A2018A0
:1001F0001302120093022000E31252FE130EC000FD
:10020000130200009300000013000000130100001F
:10021000639820161302120093022000E31452FE8A
:10022000130ED00013020000930000001300000022
:100230001301000013000000639420141302120045
:1002400093022000E31252FE130EE000130200009E
:1002500093000000130000001300000013010000D1
:10026000639020121302120093022000E31252FE48
:10027000130EF000130200009300000013010000B1
:10028000639020101302120093022000E31652FE26
:10029000130E000113020000930000001301000080
:1002A00013000000639E200C130212009302200032
:1002B000E31452FE130E100113020000930000001D
:1002C000130100001300000013000000639A200ACD
:1002D0001302120093022000E31252FE130E2001BB
:1002E000130200009300000013000000130100003F
:1002F000639820081302120093022000E31452FEB8
:10030000130E3001130200009300000013000000E0
:100310001301000013000000639420061302120072
:1003200093022000E31252FE130E4001130200005C
:1003300093000000130000001300000013010000F0
:10034000639020041302120093022000E31252FE75
:1003500093001000639A00009380100093801000B7
:100360009380100093801000938010009380100001
:10037000930E3000130E50016394D001631CC00132
:100380000F00F00F63000E00131E1E00136E1E0000
:10039000730000000F00F00F130E10007300000038
:1003A000731000C00000000000000000000000000A
:1003B000000000000000000000000000000000003D
:0403C0000000000039
:1010000000000000000000000000000000000000E0
:1010100000000000000000000000000000000000D0
:1010200000000000000000000000000000000000C0
:1010300000000000000000000000000000000000B0
:081040000000000000000000A8
:040000058000200057
:00000001FF
